:1000000008308A00E62D0000FF00030E8312031360
:10001000A1000A08A0008A010408A2007708A30032
:100020007808A4007908A5007A08A6007B08A70034
:10003000831383128B1E1E280B193128220884007B
:100040002308F7002408F8002508F9002608FA001C
:100050002708FB0020088A00210E8300FF0E7F0E78
:1000600009008A110A12CA280A108A100A11820786
:10007000533475346E344D346F346E3454347534B7
:1000800065345734653464345434683475344634D4
:100090007234693453346134743400340A108A1071
:1000A0000A11820700341E34253429341E340034EA
:1000B000003411343F3401340034113423342534F6
:1000C000193400341E34253429341E340A108A10A1
:1000D0000A118207443441345934203454344934A9
:1000E0004D34453420342034543445344D34503468
:1000F00020345034523445345334533400340A10CD
:100100008A100A1182072B343334353463340034B7
:100110000A108A100A1182072B34323430346334C7
:1001200000340A108A100A118207203430346334F4
:10013000203400340A108A100A1182072D34313419
:100140003534633400340A108A100A1182072B34C4
:1001500031343534633400340A108A100A118207AE
:100160002D3432343034633400340A108A100A11CA
:1001700082072D3433343534633400340A108A1046
:100180000A11820720342D3430342E34253475344E
:1001900020340034AD0BD0281030AD002814AE0A46
:1001A0002E083B3C0318DB28AE01AF0A2F081E3C8B
:1001B000031DDB28A8142F083B3C0318E228AF01DD
:1001C000B00A28153008183C031DE828B001B10A10
:1001D0003108063C0318ED28B1010B118A110A12EF
:1001E0001E28A9012908113C031CFD284A302907B3
:1001F0008400FF308000A90AF2288E3083169F0009
:1002000083121F083839C1389F0085018601870194
:10021000FF3083168500003086000F308700831280
:100220002810A8102811A81581010730F700F71D24
:10023000212907308101813084000008C0390F383E
:1002400080006400813084000008C0397704800099
:100250008B16C0308B048A150A12F62D5F3084008D
:100260000008031940290130F800F701F70B36297F
:10027000F80B35295B30F700F70B3C29800B33294D
:100280000034FF3083168600831287178712071306
:10029000000000000608B4000717000000008716E1
:1002A00000308316860083120034412160088600E6
:1002B000871307120713000007170716412161086B
:1002C000860087130712071300000717071600346C
:1002D00041217408860087170712071300000717CB
:1002E0000716003407168716071787170516643098
:1002F000DF002E21E101E00155214030F4006821AA
:10030000E1011430E00055214130F400682104304F
:10031000E100E00155214230F4006821E101143090
:10032000E00055214330F40068218030F40068215A
:100330009C30F40068218A150A12F92D41216008C9
:100340008600871307120713000007170716C0302F
:10035000F40068210034E101E00155212430F4006B
:100360006821B801B70138081F3C031CC329031DCD
:10037000BD293708FE3C031CC329E0019E21B70AB2
:100380000319B80AB329E101E00155212430F40032
:1003900068218A150A12012E41212030730286003D
:1003A000871307120713000007170716C030F40061
:1003B00068210034E101E00155212430F400682176
:1003C000DE015E086620DE0AF300CC2114305E02F6
:1003D000031DE1290430DF002E210530E1005430F7
:1003E000E00055212430F40068212830A900A90834
:1003F0000319FF29FF30E0009E21A903F7298A1580
:100400000A12042EF701F8015E0803105F18F707BF
:10041000F70CF80CDF18F707F70CF80C5F19F70763
:10042000F70CF80CDF19F707F70CF80C5F1AF70751
:10043000F70CF80CDF1AF707F70CF80C5F1BF7073F
:10044000F70CF80CDF1BF707F70CF80C0034620808
:10045000F801610203182F2A6108F7003B2AF7010F
:100460000830E300E10DF70D620877020318F7008A
:10047000F80DE30B322A00346018562AE018692A76
:100480005F08E1006430E20027227708DF00780887
:100490003030031D502A6019562AE0192030522AA4
:1004A0006011E011F8077808F300CC215F08E10043
:1004B0000A30E20027227708DF0078083030031D79
:1004C000652A6019692AE0192030F8077808F300D6
:1004D000CC213030DF075F08F300CC2100340B1350
:1004E0008B138B1B702A0708FF3A0F39F700013076
:1004F00077020319882A023077020319892A043007
:1005000077020319902A083077020319972A9E2A46
:100510009F2AB10A3108063C03188F2AB1019F2A8D
:10052000B00A3008173C0318962AB0019F2AAF0A78
:100530002F083B3C03189D2AAF019F2A9F2AE10107
:100540001430E00055212430F40068213108DE0029
:100550000330DF0002227808A9000330AA00AA08AD
:100560000319BA2A29083420DE00F300CC21A90A95
:10057000AA03AF2A2030F300CC213008DF0001307D
:10058000E0003C223A30F300CC212F08DF0001309C
:10059000E0003C220230DE00FA30DF002E21DE0BCC
:1005A000CC2A0030851A0130003A0319732AAE01B3
:1005B000C0308B048A150A12182EDE080319E62AA9
:1005C00085143D30831685008312EA2A3F30831656
:1005D00085008312003485103D3083168500F43089
:1005E000F7008312F70BF22A3F3083168500D130D3
:1005F000F7008312F70BFA2A000000340830DF00FE
:100600000310DE0C031C172B85103D30831685006C
:100610000330F7008312F70B0B2B3F308316850056
:100620001430F7008312F70B132B0000242B8510D6
:100630003D30831685001830F7008312F70B1E2B10
:100640003F30831685008312DF03DF08031D002B74
:1006500000345E085F068039E100DE1F312BDE09C1
:10066000DE0ADF1F352BDF09DF0A5F08F8015E02B3
:1006700003183D2B5E08F700492BF7010830E00016
:10068000DE0DF70D5F0877020318F700F80DE00B99
:10069000402BE11F4D2BF809F80A000000348E3082
:1006A000F7005F08F8005E08F900FA01F808031D7A
:1006B000632B7908F800F9010830F702F808031DE8
:1006C000632BF7016B2B0310F81B6A2BF90DF80D48
:1006D000F703632BF81300008A110A12802E5E08BC
:1006E0000319352CEA0062080319352CEA020318B5
:1006F0007A2B7F2B7F30EA070318352C852B81302E
:10070000EA02031C352C0319352C6A08F700F8019E
:10071000F901FA01E9015F08E800E8176008E7005D
:100720006108E6001930EA006508E6020318A82B04
:100730000130E7020318A82BE8020318A82BE902EE
:100740000318A82BE90AE80AE70A6508E607DA2B86
:100750006408E7020318C32B0130E8020318C32B17
:10076000E9020318C32BE90AE80A6408E7076508E9
:10077000E607031CDA2BE70A031DDA2BE80A031D40
:10078000DA2BE90ADA2B63088038E8020318D92B40
:100790000130E9020318D92BE90A63088038E80719
:1007A0006408E707031CB72BE80A031DB72BE90A07
:1007B000B72B7A14EA0BDD2BE82B0310E60DE70DBF
:1007C000E80DE90D0310FA0DF90DF80DEB0D942B62
:1007D0006B1CF02B0310F80CF90CFA0CEB0CF32B40
:1007E000F7030319352CEB1B1C2C0310E60DE70D4A
:1007F000E80DE90D6508E6020318082C0130E70250
:100800000318082CE8020318082CE902031C2B2CFF
:100810006408E7020318132C0130E8020318132CB4
:10082000E902031C2B2C63088038E80203181C2CF7
:100830000130E902031C2B2CFA0A031D2B2CF90AA8
:10084000031D2B2CF80A031D2B2CF70A0319352C3A
:10085000F80CF90CFA0C5F08EA006308EA06EA1FD4
:10086000332CF817392CF813392CF701F801F9015A
:10087000FA0100008A110A12912E80300418E30652
:10088000E8015F08E7006308E7065E0803192A2D00
:10089000E600F70062080319332DE6020319D02C95
:1008A0000318532C8F2C6308EC00EC176408EB0042
:1008B0006508EA00E9010310EC0CEB0CEA0CE90C0A
:1008C000E60B5A2CE71F672C6814472D681066103A
:1008D0006816613084005D2D6812E71B792C661C58
:1008E000842CEC0CEB0CEA0CE90CF70A0319422DF2
:1008F000842CEC1B872C0310E90DEA0DEB0DEC0D9D
:10090000F7030319422D792C6817EF2C68135F0841
:10091000E700E71F8D2CEC173B2DEC133B2D6208F5
:10092000E600F7005E08E6025F08EC00EC176008DE
:10093000EB006108EA00E9010310EC0CEB0CEA0C97
:10094000E90CE60B9B2CE71FA82CE814472DE810B8
:100950006610E816653084005D2DE812E71BBA2C9E
:10096000661CC52CEC0CEB0CEA0CE90CF70A03191D
:10097000422DC52CEC1BC82C0310E90DEA0DEB0D24
:10098000EC0DF7030319422DBA2CE817EF2CE813EE
:100990006308E700E71FCE2CEC173B2DEC133B2D33
:1009A0006308EC00EC176408EB006508EA00E71F39
:1009B000DD2CEC136815472D6811E90166106130D4
:1009C00084005D2DE71B052D5F08E700661CEF2CFA
:1009D000EC0CEB0CEA0CE90CF70A0319422DE91FA9
:1009E000002DEA0A031D002DEB0A031D002DEC0A61
:1009F000031D002DEC0CEB0CEA0CF70A0319422D39
:100A0000681B862CE81BC72C242D8030EC06EC1FBD
:100A10000D2D472D6308E7001A2D5F08E700EC084D
:100A2000031D1A2DEB08031D1A2DEA08031D1A2DAC
:100A3000F7013B2DEC1B242D0310E90DEA0DEB0D06
:100A4000EC0DF70B1A2D422DE71F282DEC173B2D2F
:100A5000EC133B2D6208F7006308EC006408EB0020
:100A60006508EA003B2D5E08F7005F08EC006008AF
:100A7000EB006108EA006C08F8006B08F9006A08EE
:100A8000FA007C2DF701F801F901FA017C2DE9014A
:100A9000EA09EB09EC09E909E90A031D562DEA0AFE
:100AA000031D562DEB0A031D562DEC0A6818662C03
:100AB000E818A72C6819DC2C0A2D0008EA07031C8B
:100AC000672DEB0A031D672DEC0A031966148403D6
:100AD0000008EB07031C6F2DEC0A0319661484034E
:100AE0000008801B742D803AEC0703186614681AFE
:100AF0006C2CE81AAD2CE22C00008A110A12A92EE7
:100B00000030F8001F08C73978049F00DE01DD229D
:100B100000000000EB22CC30DE00FE22BE30DE0002
:100B2000FE22DE01DF011030E000E0080319B22DE3
:100B300085103D30831685003F30850000000000A1
:100B400000000000000083128518A82D0310A92DB5
:100B50000314DF0CDE0C1B30F700F70BAD2D00008B
:100B6000E003952D5E08F8005F08F9007808B900E9
:100B7000EB22CC30DE00FE224430DE00FE220130CB
:100B8000DE00DD223908DE000230DF00292378088C
:100B9000BA003908DE000230DF0029237708003A66
:100BA0000319D52D0530BB00D62DBB013A08803A7C
:100BB000713C031CDC2D2812BA1BE32D3A080E3CB5
:100BC0000318E32D2816281E2B2EE1013C30E000EF
:100BD00055212430F4006821DE015E087F20DE0A02
:100BE000F300CC2104305E02031DED2DE1017830CD
:100BF000E00055212430F4006821DE015E088820E1
:100C0000DE0AF300CC2104305E02031DFE2DE1015B
:100C1000DC30E00055212430F4006821DE015E085C
:100C20009120DE0AF300CC2104305E02031D0F2E5A
:100C30000130E1001830E00055212430F400682133
:100C4000DE015E089A20DE0AF300CC2104305E0249
:100C5000031D212E702EE1013C30E000552124308F
:100C6000F4006821DE015E08A320DE0AF300CC2137
:100C700004305E02031D332EE1017830E00055217F
:100C80002430F4006821DE015E089120DE0AF300C2
:100C9000CC2104305E02031D442EE101DC30E00073
:100CA00055212430F4006821DE015E08AC20DE0A04
:100CB000F300CC2104305E02031D552E0130E1000B
:100CC0001830E00055212430F4006821DE015E0870
:100CD000B520DE0AF300CC2104305E02031D672E2E
:100CE0001F151F19712E1E08FA0083161E08831285
:100CF000B5007A08B6003608DF003508DE004F2B55
:100D00007A08E1007908E0007808DF007708DE0063
:100D10009A30E5009930E4004C30E3008530E20081
:100D20006F2B7A08BF007908BE007808BD007708ED
:100D3000BC0084013F08E1003E08E0003D08DF0000
:100D40003C08DE00E501E4013E30E3008530E200CE
:100D50003D2C7A08BF007908BE007808BD007708EE
:100D6000BC008A150A12212E5E08F700F71FC12E5B
:100D7000F709F70A7708DE002D30F800F300CC21E0
:100D8000DF0A5F18DB2EDF18EE2E5E08E10064300C
:100D9000E20027227708DE0078083030031DD52EC8
:100DA0005F19DB2EDF192030D72E5F11DF11F80716
:100DB0007808F300CC215E08E1000A30E200272227
:100DC0007708DE0078083030031DEA2E5F19EE2E1A
:100DD000DF192030F8077808F300CC213030DE0727
:100DE0005E08F300CC2100345F08E6006308E606E5
:100DF000E61FFF2E03110310DF1B0314322F5F08C1
:100E0000E6006208E7005E08E70203190D2FE61FFF
:100E1000322F0308013A8300322F6308E7005F088E
:100E2000E7020319192FE61F322F0308013A830046
:100E3000322F6408E7006008E7020319252FE61F38
:100E4000322F0308013A8300322F6508E70061085A
:100E5000E7020319312FE61F322F0308013A8300FE
:100E6000322F03108A150A124B2A0530C100903028
:100E7000C0000130A90029086C3C031CA12F4108C7
:100E8000E1004008E00055212430F40068211430CE
:100E9000AA00AA0803196F2F01302A024A3EDF0078
:100EA000E0014121C130F40068214121FF30831667
:100EB00086008312871387120713000000000608BC
:100EC000E00007178716003083168600831260083B
:100ED000F8005F08840078088000AA03492F0310F7
:100EE000CA0DCB0DCC0DCD0DCE0DCF0DD00DD10D2E
:100EF000D20DD30DD40DD50DD60DD70DD80DD90DDE
:100F0000DA0DDB0DDC0DDD0D4108E1004008E000ED
:100F100055212430F40068211430AA00AA080319CE
:100F20009B2F01302A024A3E84000008DF00E000C7
:100F30009E21AA038E2F1430C0070318C10AA90AE4
:100F40003B2F00345F0861068039E300DF1FAD2FBF
:100F5000DE09DF09DE0A0319DF0AE11FB42FE00909
:100F6000E109E00A0319E10A1030F700FA01E20191
:100F7000DF0CDE0C031CC22F6008FA070318E20A1C
:100F80006108E207E20CFA0CF90CF80CF70BB82F29
:100F9000E31FCF2FF809F909F80A0319F90A00002D
:100FA00000348E30F7005E08F7025F08F900600831
:100FB000F800F917F7080319E82F0310F908031DC3
:100FC000E42FF8080319E82FF90CF80CF70BDD2FC4
:100FD000DF1FEF2FF809F909F80A0319F90A0000D1
:060FE0008A150A12762BAF
:101000000408E700E801DF1F0A282D30F3008A11E9
:10101000CC218A15DF175E080319AE287F305E02E7
:10102000031C6928DE00ED010430EE000310E10D21
:10103000E00DDF0DE80DEE0B162804305E020318FC
:10104000292803305E02031DA3280A306802031C0E
:10105000A3280330DE02ED0A50210310E10DE00D5C
:10106000DF0DE80D39210230EE000310E80CDF0C33
:10107000E00CE10CEE0B352850210430EE0003109B
:10108000E90CEA0CEB0CEC0CEE0B3F28392150215B
:101090006B08EC006A08EB006908EA00E9013921F5
:1010A00050216A08EC006908EB00E901EA013921E6
:1010B000E8191D28DE08031D6228E10AE00ADF0A9C
:1010C000E80AA3280310E10DE00DDF0DE80DDE03B3
:1010D0001D28DE09DE0A7F30DE07ED010430EE0058
:1010E0000310E10DE00DDF0DE80DEE0B702804306C
:1010F000DE0705305E02031CB02850210310E10D0D
:10110000E00DDF0DE80D0310E10DE00DDF0DE80D42
:1011100039210310E10DE00DDF0DE80DED0A03307C
:10112000EE000310E80CDF0CE00CE10CEE0B912854
:101130000330DE02681E79280310E80CDF0CE00C97
:10114000E10CDE037928DE09DE0A0330DE076D08D4
:10115000E3006D08E500670AE507DD28670AED0092
:101160003030F3008A11CC218A15E708031937299A
:101170002E30F3008A11CC218A156D08E600E603B3
:1011800067086602031CC6286708E600E60803191C
:10119000D0283030F3008A11CC218A15E60BC928FB
:1011A0006D08EE00670AEE0203185929DE03670A8C
:1011B000E5006D08E5026508E3006808E2005E08E6
:1011C0000319E728E4000310E20CE40BE3286508A8
:1011D0000319372930306207F3008A11CC218A15B0
:1011E0006308031DFB28E708031937292E30F30095
:1011F0008A11CC218A15E303E503031937295E0818
:1012000003190729E4000310E20DE40B0329620827
:10121000E8026808E9005F08EA006008EB0061087E
:10122000EC000310E10DE00DDF0DE80D0310E10D02
:10123000E00DDF0DE80D6C08E107031C2429E00F29
:101240002429DF0F2429E80A6B08E007031C2B2957
:10125000DF0F2B29E80A6A08DF070318E80A690884
:10126000E8070310E10DE00DDF0DE80DDD280000BB
:1012700059296C08E107031C4229E00F4229DF0FBE
:101280004229E80A6B08E007031C4929DF0F4929B6
:10129000E80A6A08DF070318E80A6908E807003463
:1012A0006808E9005F08EA006008EB006108EC00EC
:1012B000003400000034E1011430E0008A115521AF
:1012C0008A152430F4008A1168218A153108DE005D
:1012D0000330DF008A1102228A157808A900033042
:1012E000AA00AA080319802929088A1134208A151E
:1012F000DE00F3008A11CC218A15A90AAA037129FC
:101300002030F3008A11CC218A153008DF0001302B
:10131000E0008A113C228A153A30F3008A11CC2170
:101320008A152F08DF000130E0008A113C228A155F
:10133000B91BBC293908133C0318BC292030F30021
:101340008A11CC218A153A08DE000C30DF008A11A0
:10135000B4268A152E30F3008A11CC218A153B0859
:10136000DF000C30E0008A113C228A152030F300A7
:101370008A11CC218A153B2AB91BE1292030F300C0
:101380008A11CC218A152030F3008A11CC218A15CC
:101390003A08DE000C30DF008A11B4268A152E30A0
:1013A000F3008A11CC218A153B08DF000C30E000E5
:1013B0008A113C228A152030F3008A11CC218A152B
:1013C0003B2A3908FF3C031D002ADE015E088A1112
:1013D000BE208A15DE0AF3008A11CC218A1504305A
:1013E0005E02031DE6293B08DF000C30E0008A1195
:1013F0003C228A152030F3008A11CC218A153B2A21
:101400003908803A6C3C031C1E2A3A08DE000C3076
:10141000DF008A11B4268A152E30F3008A11CC2100
:101420008A153B08DF000C30E0008A113C228A1547
:101430002030F3008A11CC218A153B2A2030F3009A
:101440008A11CC218A153A08DE000C30DF008A119F
:10145000B4268A152E30F3008A11CC218A153B0858
:10146000DF000C30E0008A113C228A152030F300A6
:101470008A11CC218A153F08E1003E08E0003D08B2
:10148000DF003C08DE00E501E4014830E300853080
:10149000E2008A11F42E8A15031C5F2A2030F30023
:1014A0008A11CC218A15013084003F08E1003E08F2
:1014B000E0003D08DF003C08DE0000206A2A013021
:1014C00084003F08E1003E08E0003D08DF003C08E2
:1014D000DE0000200030A8190130013C031D802AE5
:1014E000E1011A30E0008A1155218A152430F400F8
:1014F0008A1168218A152A30F3008A11CC218A15B5
:101500000030A8190130FF3E003A031D892AA811B6
:101510008A2AA8158A150A12232E5E080319FE2AA4
:10152000E60062080319FE2AE607031C982A9F2A90
:101530007F30E602031CFE2A0319FE2AA32A81300B
:10154000E6070318FE2A6608F700F801F901FA0118
:101550005F08EA00EA176008E9006108E80018304F
:10156000E600E701681CCC2A6508FA07031CBE2ABE
:10157000F90A031DBE2AF80A0319E7176408F907D8
:10158000031CC52AF80A0319E7176308E000E017EF
:101590006008F8070318E717E70DF80CF90CFA0CC8
:1015A000EA0CE90CE80C0310E60BB12A0130F7074E
:1015B0000318FE2AF81BE32AEA0DFA0DF90DF80DBF
:1015C000F7030319FE2AEA1FF42AFA0A031DF42A74
:1015D000F90A031DF42AF80A031DF42AF80CF90C81
:1015E000FA0CF70A0319FE2A5F08E7006308E7060A
:1015F000E71FFC2AF817022BF813022BF701F8015A
:10160000F901FA0100008A150A126C2B0030281A21
:101610000130003A031D132B46303907C400C501C1
:10162000C41BC503192B1E303907C400C501C41BD8
:10163000C503C51F1C2B1D2B1F2BC501C401C51BBA
:101640002B2BC508031D282B4408643C03182B2BA7
:10165000C5016430C4004408643CC4000030F80094
:101660004508031C450F362B7808372B7802C50038
:101670004508DF004408DE00E1011430E0008A1173
:10168000A2278A157908C5007808C400A330C407CA
:101690000318C50A0530C5074508E1004408E00005
:1016A0008A1155218A152430F4008A1168218A157F
:1016B000F830F4008A1168218A153F08E1003E08DD
:1016C000E0003D08DF003C08DE00E501E4012030D9
:1016D000E3008230E2008D2A7A08E1007908E00018
:1016E0007808DF007708DE008A11D12F8A15790883
:1016F000C5007808C400B630C4020330031C0430AF
:10170000C502C51F842B852B872BC501C401C51BB2
:10171000932BC508031D902B4408643C0318932B9E
:10172000C5016430C4004408643CC4000030F800C3
:101730004508031C450F9E2B78089F2B7802C50097
:101740004508DF004408DE00E1011430E0008A11A2
:10175000A2278A157908C5007808C400A330C407F9
:101760000318C50A0530C5074508E1004408E00034
:101770008A1155218A152430F4008A1168218A15AE
:10178000F830F4008A1168218A1514304407DE000D
:101790004508DF000318DF0A5F08E1005E08E0008B
:1017A0008A1155218A152430F4008A1168218A157E
:1017B000F830F4008A1168218A1500341030F700DF
:1017C000FA01E201DF0CDE0C031CEC2B6008FA07C7
:1017D0000318E20A6108E207E20CFA0CF90CF80CB3
:1017E000F70BE22B00343008153C031CFB2B3008B0
:1017F000023C031C492C32088A114E208A15F8003D
:10180000B3000D30C500FF30C400C701C601C708D2
:10181000031D482C4608053C031C482CDF011430EE
:10182000DE004708E1004608E000DE237908FA0000
:1018300078084402DE004508DF007A08031C7A0FAE
:10184000DF025F08E1005E08E0008A1155218A1579
:101850002430F4008A1168218A153308F7004608FD
:10186000F8000319372C0310F70CF80B332C771CF6
:101870003F2CF830F4008A1168218A15442CF0308E
:10188000F4008A1168218A15C60A0319C70A072CB1
:10189000B20A3008093C03189F2C30080E3C031C88
:1018A0009F2C32088A114E208A15F800B3000D30A3
:1018B000C500FF30C400C701C601C708031D9E2C28
:1018C0004608053C031C9E2CDF011430DE0047084F
:1018D000E1004608E000DE237908FA0078084402B7
:1018E000DE004508DF007A08031C7A0FDF025F087C
:1018F000E1005E08E0008A1155218A152430F400C9
:101900008A1168218A153308F7004608F800031980
:101910008D2C0310F70CF80B892C771C952CF830C4
:10192000F4008A1168218A159A2CF030F4008A118B
:1019300068218A15C60A0319C70A5D2CB20A003449
:101940003008F700F7080319B22C063077020319A4
:10195000E32C0C3077020319152D1230770203198E
:10196000472D792DB2010530C500A330C400C70151
:10197000C6014708073C031CE22C031DC32C460884
:10198000D03C031CE22C46084407DE004508DF007B
:101990000318DF0A4708DF075F08E1005E08E00080
:1019A0008A1155218A152430F4008A1168218A157C
:1019B000F830F4008A1168218A152830C607031808
:1019C000C70AB92C7A2D0630B2000530C500A33005
:1019D000C400C701C6014708073C031C142D031DA2
:1019E000F52C4608D03C031C142D46084407DE00A5
:1019F0004508DF000318DF0A4708DF075F08E1003A
:101A00005E08E0008A1155218A152430F4008A11FD
:101A100068218A15F830F4008A1168218A15C830C7
:101A2000C6070318C70AEB2C7A2D0A30B20005301E
:101A3000C500A330C400C701C6014708073C031C0A
:101A4000462D031D272D4608D03C031C462D460875
:101A50004407DE004508DF000318DF0A4708DF07F8
:101A60005F08E1005E08E0008A1155218A152430E4
:101A7000F4008A1168218A15F830F4008A1168216F
:101A80008A156430C6070318C70A1D2D7A2D103039
:101A9000B2000530C500A330C400C701C601470825
:101AA000073C031C782D031D592D4608D03C031C10
:101AB000782D46084407DE004508DF000318DF0ADA
:101AC0004708DF075F08E1005E08E0008A11552142
:101AD0008A152430F4008A1168218A15F830F40040
:101AE0008A1168218A15C830C6070318C70A4F2D06
:101AF0007A2D7A2D30080139003A031DE32D053087
:101B0000C500A330C400C701C6014708023C031C3E
:101B1000B02D031D8F2D4608583C031CB02D4608E0
:101B20004407DE004508DF000318DF0A4708DF0727
:101B30005F08E1005E08E0008A1155218A15243013
:101B4000F4008A1168218A15F830F4008A1168219E
:101B50008A155830C6070318C70A0230C707852DF3
:101B60007830C4070318C50A0530C507C701C60188
:101B70004708023C031CE32D031DC22D4608583CB8
:101B8000031CE32D46084407DE004508DF00031868
:101B9000DF0A4708DF075F08E1005E08E0008A11FE
:101BA00055218A152430F4008A1168218A15F830ED
:101BB000F4008A1168218A155830C6070318C70A2D
:101BC0000230C707B82D8A150A123B2E84011F3038
:101BD000830583169F01831228160830AD00AE01DD
:101BE000AF01B001B101B2018A11F1288A158A1141
:101BF00072298A15C830DF008A112E218A158A11B0
:101C0000AB298A158A11DA298A150030851A013024
:101C1000003A031D192E1930DF008A112E218A1572
:101C20000030851A0130003A031D192E8A116F2ADF
:101C30008A15003028180130013C031D242E8A111A
:101C4000802D8A155B2928100030A8180130013C2E
:101C5000031D302E8A1135278A150623F323A81079
:101C6000003028190130013C031D3D2E8A11352713
:0E1C70008A150623A02CF3232811052E6300ED
:02400E00410D62
:00000001FF
